:100000000C944A030C9482030C9482030C94820394
:100010000C9482030C9482030C9482030C9482034C
:100020000C9482030C9482030C94F52A0C94C72B35
:100030000C94D4250C9482030C9482030C948203B8
:100040000C9482030C9482030C9482030C9482031C
:100050000C941C200C945C260C9482030C94820358
:100060000C9482030C9482030C9482030C948203FC
:100070000C9482030C9482030C9482030C948203EC
:100080000C9482030C9482030C9482030C948203DC
:100090000C9482030C9482030C9482030C948203CC
:1000A0000C9482030C9482030C9482034E064E0639
:1000B0007A067A06E2060007180818080B07A40754
:1000C000B507B5072B1F2D1F321F351F381F3B1FCC
:1000D0003E1FDD22D322E02228232C232C23282399
:1000E0002C232C2301232C230B2315232C232C23FB
:1000F0002C232C2328232C232C2328232C23EE22CF
:100100002C232C23252325232523252325232523A1
:100110002523252325232A232C23DD22D0222C232B
:100120002C232C232C232C232C232C232C232C2357
:100130002C232A232C232C2328232C23232323235F
:1001400023232323232323232323232323232A2378
:10015000342C5B2C532D5B2C532DA72CCA2C532DE8
:10016000212D302D29001E001F002000210022001B
:10017000230024002500260027002D002E002A0041
:100180002B0014001A000800150017001C001800AE
:100190000C00120013002F00300031000151040048
:1001A0001600070009000A000B000D000E000F00EA
:1001B000330034004C002800E10031001D001B001A
:1001C0000600190005001100100036003700380045
:1001D000E5004C00E000E300E20000002C0000001D
:1001E0002C0000002C000000E600E7006500E400A1
:1001F000005C3A003B003C003D003E003F004000F8
:10020000410042004300440045004C000100010051
:100210004B0001000100010001000100520001003B
:10022000AC00AE00AB00C15C01004A004E004D00C6
:100230000100AA00A900500051004F000100010078
:100240002A00010001000100C35CC45CC65CC75CFD
:10025000C85CC95CCA5CCB5C0100010046000100BF
:100260000100010001000000010000000100000089
:1002700001000000010001000100010000047F3FB7
:100280001F643214643214783C1E1E140A052223A3
:10029000252628292A2C2D2F3032333536383A3B63
:1002A0003D3E4042434547494A4C4E5051535557B5
:1002B000595A5C5E6062646668696B6D6F717375D4
:1002C00077797B7D7F81838587898A8C8E909294D4
:1002D00096989A9C9E9FA1A3A5A7A8AAACAEAFB1E1
:1002E000B3B4B6B8B9BBBCBEBFC1C2C3C5C6C7C92B
:1002F000CACBCCCDCED0D1D2D2D3D4D5D6D7D7D8E5
:10030000D9D9DADADBDBDBDCDCDCDCDCDDDDDDDD36
:10031000DCDCDCDCDCDBDBDBDADAD9D9D8D7D7D63E
:10032000D5D4D3D2D2D1D0CECDCCCBCAC9C7C6C5F5
:10033000C3C2C1BFBEBCBBB9B8B6B4B3B1AFAEAC3B
:10034000AAA8A7A5A3A19F9E9C9A98969492908EE6
:100350008C8A89878583817F7D7B79777573716FBF
:100360006D6B6968666462605E5C5A59575553519B
:10037000504E4C4A4947454342403E3D3B3A383651
:10038000353332302F2D2C2A292826252322FFAA67
:100390007F55400000000000000000000000010147
:1003A0000203040506080A0C0F1114181C20242946
:1003B0002E33393F464C535B626A7179818A929A37
:1003C000A2AAB2B9C1C8CFD5DCE1E7EBF0F4F7FAE5
:1003D000FCFDFEFFFEFDFCFAF7F4F0EBE7E1DCD5F7
:1003E000CFC8C1B9B2AAA29A928A8179716A625BB6
:1003F000534C463F39332E2924201C1814110F0C5E
:100400000A080605040302010100000000000000C4
:1004100000000000010101010101010101020202CD
:1004200002020202020203030303030303030404A0
:10043000040404040405050505050606060606076A
:100440000707070708080808090909090A0A0A0B23
:100450000B0B0C0C0C0D0D0D0E0E0E0F0F0F1010C4
:10046000111111121213131414151516161717184B
:100470001819191A1A1B1B1C1D1D1E1E1F202021B6
:100480002222232424252626272829292A2B2C2DFD
:100490002D2E2F30313232333435363738393A3B1E
:1004A0003C3D3E3F404142434445464748494A4C13
:1004B0004D4E4F50515354555658595A5B5D5E5FDF
:1004C000616264656668696B6C6D6F707273757775
:1004D000787A7B7D7E8082838587888A8C8E8F91D7
:1004E000939596989A9C9EA0A2A3A5A7A9ABADAF01
:1004F000B1B3B5B7BABCBEC0C2C4C6C9CBCDCFD1EB
:10050000D4D6D8DBDDDFE2E4E7E9EBEEF0F3F5F893
:10051000FAFDFF100350006F006C0061007200696B
:1005200000730000002603610069003000330020E2
:1005300000440065007300690067006E00200053EE
:100540000074007500640069006F00000004030976
:100550000409023B00020100A0FA090400000103A3
:10056000010100092111010001224000070581035A
:100570000800010904010001030000000921110124
:10058000000122B6000705820320000112010002CB
:100590000000000803A102000100010200010501A2
:1005A0000902A10185020901A10005091901290813
:1005B00015002501950875018102050109300931F1
:1005C0001581257F95027508810609381581257FDB
:1005D000950175088106050C0A38021581257F955D
:1005E0000175088106C0C005010980A101850319B4
:1005F000012AB700150126B700950175108100C0CA
:10060000050C0901A101850419012AA00215012682
:10061000A002950175108100C005010906A10185A0
:1006200006050719E029E7150025019508750181E0
:10063000020507190029EF1500250195F0750181C4
:1006400002050819012905950575019102950175A5
:10065000039101C005010906A101050719E029E779
:100660001500250195087501810295017508810124
:100670000507190029FF150026FF0095067508815A
:100680000005081901290595057501910295017567
:10069000039101C011241FBECFEFDAE0DEBFCDBF52
:1006A00004B603FE18C080913D0390913E03A091D3
:1006B0003F03B09140038730904BA740B04B59F4B3
:1006C00010923D0310923E0310923F03109240039C
:1006D000E0E0F8E3099511E0A0E0B1E0ECE2FDE52F
:1006E00002C005900D92A83CB107D9F723E0A8EC11
:1006F000B1E001C01D92AD33B207E1F70E942A14A8
:100700000C94942E0C94000081E0089581E00895EB
:100710000C94860308950C948A031F93CF93DF9360
:1007200000D000D01F92CDB7DEB749835A836B83C8
:100730003091CB0189819A81311114C0662359F01F
:10074000222349F00E94550A182F682F89819A8127
:100750000E94FE0903C00E94290A182F69817A812C
:10076000812F04C00E94550A69817A810F900F90F1
:100770000F900F900F90DF91CF911F910C949511D6
:10078000FC01262F408151816281738184810C9408
:100790008D0381E00895CF93DF93EC0160E00E9428
:1007A000C003BE01DF91CF910C948B030C94DB123C
:1007B0000C94D71208950E94A8080E94DA032FEF24
:1007C00084E39CE0215080409040E1F700C00000AD
:1007D0000C9482260F931F93CF93DF938C0161E0DB
:1007E0000E94C003EC01B8010E948803882309F429
:1007F0004BC0B801CE010E941C1F882309F444C0DD
:10080000B801CE010E941F248823F1F1B801CE0166
:100810000E94E3208823C1F1B801CE010E947B230E
:10082000882391F1B801CE010E94331D882361F124
:10083000F8018281882309F1CB358DE5D807C1F015
:1008400050F4C115FCE5DF0781F0CF3DDC45A9F48C
:100850000E948C0F19C0CC35EDE5DE0761F0CD3577
:10086000DD4559F40E94CF0E08C00E94DB030CC086
:100870000E94D80E02C00E94DB0EC801DF91CF910A
:100880001F910F910C94840380E0DF91CF911F9111
:100890000F9108950E94B62580E00E94D41F0E9407
:1008A0006C040C94B01B0E94401E0E946F040E94B6
:1008B0007C1C0C94BC2508950C945B0481E0089585
:1008C0000C945E040895CF93C82F0E945C048C2F73
:1008D0000E946004CF91089580E00C9463040E940C
:1008E0007B240C9463040E947B249091CA01891795
:1008F00021F08093CA010C9463040895CF93DF9391
:10090000CDB7DEB72B970FB6F894DEBF0FBECDBFC5
:100910004F83588769877A878B8761110E941B0EE6
:100920009E012F5F3F4F86E0F90111928A95E9F70A
:1009300085E0FE013796D90101900D928A95E1F785
:1009400089819A814C815D81452B31F09F3F31F443
:1009500091E08F3F19F403C091E001C090E090FF57
:1009600009C049815A816B817C818D819E810E9461
:100970003C0D05C0C9010E94C9038111F2CF2B961D
:100980000FB6F894DEBF0FBECDBFDF91CF910895B3
:10099000FC01808191810E94970A0895CF9388235A
:1009A00009F4A9C0C82F8238C1F40E947B2481FDBC
:1009B000A2C069E380910201909103010E94712518
:1009C0000E943D0E2FEF81EE94E021508040904038
:1009D000E1F700C0000069E319C0833801F50E9407
:1009E0007B2480FD88C063E5809102019091030122
:1009F0000E9471250E943D0E2FEF81EE94E0215060
:100A000080409040E1F700C0000063E58091020162
:100A1000909103010E947C25CF910C943D0E843867
:100A2000C1F40E947B2482FD66C067E480910201CC
:100A3000909103010E9471250E943D0E2FEF81EEDF
:100A400094E0215080409040E1F700C0000067E44E
:100A5000DDCF8CEF8C0F813AF8F48C2F0E9432237B
:100A6000811149C06C2F80910201909103010E9475
:100A7000F124882349F06C2F8091020190910301A9
:100A80000E947C250E943D0E6C2F80910201909166
:100A900003010E947125C0CF80E28C0F883048F49A
:100AA000C77081E001C0880FCA95EAF70E94FE0D69
:100AB000B3CFEBE5EC0FE33040F4F0E0E45AFE4F47
:100AC000808190E0CF910C94AF24E8E5EC0FE73102
:100AD00050F4F0E0EE0FFF1FE25DFE4F8081918148
:100AE000CF910C94C524CD3E30F08C2F0E94AF14D2
:100AF000CF910C948115CF910895882309F464C097
:100B0000823879F40E947B2481FF5EC069E3809182
:100B10000201909103010E9471250E943D0E69E33C
:100B200010C08338B1F40E947B2480FF4DC063E580
:100B300080910201909103010E9471250E943D0E57
:100B400063E580910201909103010E947C250C9441
:100B50003D0E843879F40E947B2482FF35C067E41F
:100B600080910201909103010E9471250E943D0E27
:100B700067E4E7CF9CEF980F913A10F4682FE1CF2C
:100B800090E2980F983050F4877091E001C0990F6F
:100B90008A95EAF7892F0E94040ED9CF9BE5980F1A
:100BA000933020F480E090E00C94AF2498E5980F07
:100BB000973120F480E090E00C94C5248D3E20F025
:100BC0000E940A150C94811508951F93CF93DF930B
:100BD000182FEB010E94CE04209741F08FE99FE08F
:100BE0000197F1F700C000002197F6CF812FDF9128
:100BF000CF911F910C947D05893319F060E070E06E
:100C000002C060E570E00C94E505882321F00E94A5
:100C1000FE0D0C943D0E0895882321F00E94040ED1
:100C20000C943D0E0895CF92DF92EF92FF920F93B6
:100C30001F93CF93DF937C01D62FC72FFC01128126
:100C4000058102950F700E94F40D8823B9F01123DD
:100C5000A9F08C2F807F803421F080E28D0F8830C6
:100C600068F08091E70282FD09C082E00E949D0E3B
:100C70000E94F40D91E0D82ED92601C0D12CCC2EA3
:100C8000C2948FE0C8228C2D90E08C30910508F042
:100C9000CFC1FC01EA5AFF4F0C94EF2D8C2F807FBF
:100CA000CF70882311F0C295C07F112399F0CC2317
:100CB00009F4AAC180E28D0F883010F0D11104C070
:100CC0008C2F0E94FE0D03C08C2F0E940E0E0E94DE
:100CD0003D0E9AC18D2F0E947D05CC2309F4A8C139
:100CE00080E28D0F883038F1DD2329F18C2F0E94AE
:100CF000140E24C08C2F807FCF70803211F0C295EB
:100D0000C07FDD2319F0D130A1F13DC08091E70211
:100D100082FF17C0112349F0CC2329F08C2F0E94A9
:100D2000FE0D0E943D0E80E070C180E00E947D05B6
:100D3000CC2309F47DC18C2F0E94040E0E943D0E2D
:100D400077C1112371F0002341F0013031F40E948A
:100D50001E0E8C2B0E94260E6BC10E941E0E8C2B29
:100D60001DC0002319F0013009F462C10E94330E46
:100D700025C0112321F0063008F05AC10EC00530FD
:100D800008F056C11BC0112361F0002331F0F701B8
:100D9000858180FF39C18F7085838C2F0E94050665
:100DA00047C1002359F0D93309F03FC1FFEF07EEE7
:100DB00013E0F15000401040E1F735C18C2F0E9444
:100DC0000C0636C18C2F86958695837019F081307C
:100DD00061F02EC1112321F08D2F9C2F937002C042
:100DE00080E090E00E94AF242BC1112321F08D2FD1
:100DF0009C2F937002C080E090E00E94C52420C127
:100E00008D2F112319F00E94AF1402C00E940A1501
:100E10000E94811515C18C2F837009F047C01111F4
:100E20000BC12D2F229526952770220F220F6D2F93
:100E30006F70862F90E0A0E0B0E0022E04C0880F13
:100E4000991FAA1FBB1F0A94D2F7D4FF10C04FE00E
:100E500050E060E070E004C0440F551F661F771F2C
:100E60002A95D2F7409550956095709503C040E063
:100E700050E0BA01C695C695C3708A019B01082B44
:100E8000192B2A2B3B2BC901B801C23049F058F469
:100E9000C13019F00E941409CFC00E940209CCC0D1
:100EA0000E942609C9C00E940009C6C0112319F07A
:100EB0008C2F817001C08695882309F4BDC02D2F29
:100EC000229526952770220F220F6D2F6F70862F87
:100ED00090E0A0E0B0E0022E04C0880F991FAA1F86
:100EE000BB1F0A94D2F7D4FF10C04FE050E060E07F
:100EF00070E004C0440F551F661F771F2A95D2F774
:100F0000409550956095709503C040E050E0BA015F
:100F1000C695C695C3708A019B01082B192B2A2BF5
:100F20003B2BC901B801C23049F058F4C13019F067
:100F30000E94D90981C00E94C7097EC00E94EB09A6
:100F40007BC00E943A0978C0CF70112339F08C2FF2
:100F50000E9460098D2F0E9405066EC08D2F0E9491
:100F60000C068C2F0E94810967C0D23F21F128F422
:100F7000D03F41F0D13FC1F043C0D33F19F1D43F3E
:100F800079F03EC0112341F0053008F051C08C2F9C
:100F90008F710E94A6094CC0063008F049C0F7CFF7
:100FA0008091E70282FF18C0112339F08C2F8F71D6
:100FB0000E9460093DC01123C9F38C2F8F710E94DC
:100FC000810936C0112329F08C2F8F710E944B09A3
:100FD0002FC00E9446092CC0112349F0CF718C2FDD
:100FE0000E94600963E08C2F0E94820E21C081E084
:100FF0000E949D0E0230E0F082E00E949D0E18C01B
:10100000112331F0002391F28D2F0E94CE0410C0E5
:10101000002399F2D93349F41FEF27EE33E0115042
:1010200020403040E1F700C000008D2F0E947D0578
:1010300088EF8C0D843020F40E947B240E9463048E
:10104000DD20C9F00E94F00D80FD15C0F70112826D
:101050000E94EA0D0E946009C7010E945C080E947C
:10106000EA0DDF91CF911F910F91FF90EF90DF90EC
:10107000CF900C948109DF91CF911F910F91FF9038
:10108000EF90DF90CF9008950F931F93CF93DF934E
:10109000EC01688179818A810E94A20A8C010E94F8
:1010A000FD090E94EE08B801CE010E941306DF91EF
:1010B000CF911F910F910895CF93DF93EC01988109
:1010C00089812B813C81232B31F08F3F31F481E0EA
:1010D0009F3F19F403C081E001C080E080FD1DC086
:1010E000CE010E94EA03811110C00E94F40D8823F2
:1010F000A1F08A81882389F08091E70282FD0DC0EA
:1011000082E0DF91CF910C949D0ECE010E944408A5
:10111000CE01DF91CF910C94CB03DF91CF91089555
:1011200080E090E00E94AF2480E090E00E94C5241F
:101130000E941B0E0E943D0E0E94B2160C94811557
:1011400080910201909103010E9487250C949008E0
:101150000E940B0E0C94A00892959F70963079F027
:1011600010F4925001C09A50923068F4803F69F0B8
:1011700018F4883E40F409C0843F29F406C0883E34
:1011800020F0813F11F080E0089581E00895FC0196
:10119000808191810E94970A0E94AC080895CF93A4
:1011A000DF9300D000D01F92CDB7DEB70F900F9025
:1011B0000F900F900F90DF91CF910895CF93DF9311
:1011C00000D000D000D0CDB7DEB726960FB6F89489
:1011D000DEBF0FBECDBFDF91CF9108950895089572
:1011E0000C94EF080C94F0080E94F2086093FD0143
:1011F0007093FE018093FF01909300020C9490087D
:101200000C94F4080F931F930091FD011091FE01BF
:101210002091FF0130910002602B712B822B932BC8
:101220001F910F910C94F4080F931F930091FD01EF
:101230001091FE012091FF01309100026023712383
:10124000822393231F910F910C94F4080F931F9303
:101250000091FD011091FE012091FF0130910002EB
:1012600060277127822793271F910F910C94F40810
:101270000C94EF080E9438096093F9017093FA0109
:101280008093FB019093FC010C94900860E070E067
:10129000CB010C943A090F931F9341E050E060E0BA
:1012A00070E08A019B0104C0000F111F221F331F31
:1012B0008A95D2F7C901B8011F910F910C943A0990
:1012C0000F931F9341E050E060E070E004C0440FD2
:1012D000551F661F771F8A95D2F78091F90190916B
:1012E000FA01A091FB01B091FC018A019B01082B3E
:1012F000192B2A2B3B2BC901B8011F910F910C947C
:101300003A090F931F9341E050E060E070E004C0A1
:10131000440F551F661F771F8A95D2F74095509549
:10132000609570958091F9019091FA01A091FB016F
:10133000B091FC018A019B01082319232A233B2336
:10134000C901B8011F910F910C943A090F931F9393
:1013500041E050E060E070E004C0440F551F661F9C
:10136000771F8A95D2F78091F9019091FA01A091A7
:10137000FB01B091FC018A019B01082719272A274C
:101380003B27C901B8011F910F910C943A090F93A3
:101390001F930091F9011091FA012091FB01309106
:1013A000FC01602B712B822B932B1F910F910C94BE
:1013B0003A090F931F930091F9011091FA012091BE
:1013C000FB013091FC0160237123822393231F9141
:1013D0000F910C943A090F931F930091F90110910A
:1013E000FA012091FB013091FC01602771278227CF
:1013F00093271F910F910C943A0908952EE0929F24
:10140000800D1124E82FE695E695E695877051E06A
:1014100001C0550F8A95EAF785E0E89FF001112495
:10142000E453FE4F20E030E070E04081CB01022E1B
:1014300002C0969587950A94E2F78170819584277A
:101440008523842781932F5F3F4F2530310569F72E
:1014500008952EE0929F800D1124682F6695669561
:101460006695982F977085E0689FB001112440E041
:1014700050E080E0FB01E40FF51FE453FE4F2081B4
:1014800030E0092E02C0369527950A94E2F72170C4
:101490003327042E01C0220F0A94EAF7822B4F5FF4
:1014A0005F4F4530510531F70895BF92CF92DF92DB
:1014B000EF92FF920F931F93CF93DF938C01C09015
:1014C000F901D090FA01E090FB01F090FC018091CD
:1014D000FD019091FE01A091FF01B0910002C82A88
:1014E000D92AEA2AFB2ACFE1D0E0D701C6010C2E87
:1014F00004C0B695A795979587950A94D2F780FD75
:1015000004C0219790F7B12C07C0BC2EB8018C2FD6
:101510000E94A8110197A9F38B2DDF91CF911F9104
:101520000F91FF90EF90DF90CF90BF900895CF93F1
:10153000DF93EC010E94550ABE010E94A811DF91C1
:10154000CF9108951F93CF93DF93EB019091CB013F
:10155000992321F0CB010E94970A13C0882349F0F8
:10156000CB010E94550A182F682FCE010E94FE0958
:1015700004C0CB010E94290A182FBE01812F0E94AE
:10158000A811DF91CF911F9108951F93CF93DF93FF
:10159000C091010216E080910202C81799F0D0E0D4
:1015A0001C9FF0011D9FF00D1124ED5FFD4F408148
:1015B000518162817381848195810E94DE08219628
:1015C000C770E9CFDF91CF911F9108954091330209
:1015D0005091340260913502709136028091370249
:1015E000909138020C94DE08EF92FF920F931F93B4
:1015F000CF93DF938091380282958F7009F065C098
:1016000080913502882309F460C080910102F09036
:1016100002021091330200913402609136027091FF
:10162000370291E01F3F09F090E0C0910001D09196
:101630000101292F96E0E92E8F1509F446C06115A6
:10164000710521F00F3F21F030E003C031E001C00F
:10165000322F90E030FD36C0E89EF001E99EF00D9B
:101660001124DF01AD5FBD4F11963C9111973013EE
:1016700029C03C91311326C012963C91129731112A
:1016800021C013964D915C911497461B570B4C1734
:101690005D07C0F4809138028F70806180933802BA
:1016A000E85FFD4F80818F708061808383E392E0EB
:1016B0000E945C08DF91CF911F910F91FF90EF90F6
:1016C0000C94C50A01968770B7CFDF91CF911F9117
:1016D0000F91FF90EF9008959F92AF92BF92CF929B
:1016E000DF92EF92FF920F931F93CF93DF93CDB7CB
:1016F000DEB761970FB6F894DEBF0FBECDBF8C0189
:1017000085E0F801DE011D9601900D928A95E1F7C2
:10171000D8011296EC9090913302E091340220911E
:101720003602309137022115310531F0EF3F31F4A7
:1017300081E09F3F19F403C081E001C080E0B82F31
:10174000B1709B2E80FD47C1D8014C9111965C91E0
:1017500011971396AD90BC90149783E3C82E82E046
:10176000D82EF0903502B501621B730B2091000159
:1017700030910101FF2009F4D9C08091380262172D
:10178000730708F095C0282F207F09F052C05E1320
:1017900013C0491311C0FE2CE1100EC08F70806180
:1017A000809338020E94E60AC6010E945C0880917C
:1017B0003802F80185834DC1AB2831F05F3F31F429
:1017C00081E04F3F19F403C081E001C080E080FD5B
:1017D00003C081E08E2502C080E090E0F82FF17018
:1017E000FF2E80FF1CC0809101022091020236E092
:1017F000821709F40BC190E0389FF001399FF00D7A
:101800001124ED5FFD4F6181561306C060814613C0
:1018100003C06281E61203C001968770E9CFFE2CF7
:10182000EE2009F416C1809138028160809338025D
:1018300054C05E1306C0491304C0E11002C0F80191
:1018400099C0C8010E94C708882361F1EE2051F1B8
:1018500020913802822F82958F7090E0029774F069
:10186000809133029091340298878F831986BB86CA
:10187000AA862C87CE0107960E945C0886E0F801B4
:10188000A3E3B2E001900D928A95E1F70E94F40A79
:101890000E94E60A0AC05E1711F1C8010E94C7083B
:1018A00081112CC0C8010E945C08FF24F394D1C0B0
:1018B000282F207F81F77A2DB98AA88A6E2D8989F1
:1018C0000E94CF0883E392E00E945C0886E0D60184
:1018D0001D928A95E9F70E94E60AF12CBAC04913D5
:1018E000DCCFE110DACFF8018583C8010E945C08E3
:1018F00086E0D6011D928A95E9F7ABC0EE2091F201
:1019000020913802822F82958F7090E002970CF41C
:10191000B5CF80913302909134029A8389831B82E0
:10192000BD82AC822E83CE010196A6CF62177307CB
:1019300008F044C0FE2CEE2009F4B4CF5E1330C092
:1019400049132EC02091380220FD21C0822F82959C
:101950008F70482F50E041155105C9F0F8012583DB
:101960004F30510541F08F5F982F9295907F822FD5
:101970008F70892B8583C8010E945C0886E0F8017E
:10198000A3E3B2E001900D928A95E1F73CC086E0B6
:10199000F801A3E3B2E001900D928A95E1F759C0F6
:1019A000C8010E94C708811169CF80913802816007
:1019B00080933802C8010E945C084BC07A2DB98A16
:1019C000A88A6E2D89890E94CF0886E0D6011D92D3
:1019D0008A95E9F718C0EE2009F464CFC8010E9487
:1019E000C708F82E882309F45DCF86E0F801A3E349
:1019F000B2E001900D928A95E1F783E392E00E94B4
:101A0000C8040E94F40A0E94E60A23C04D875E873C
:101A10008D859E850E94970A292F22952F7022304E
:101A200028F49F7039F0811105C00BC0243028F4D0
:101A30009F7049F4805E883020F0C8010E945C08E5
:101A40009F2CF92C06C0D80115969C91907F91F798
:101A5000F8CF8F2D61960FB6F894DEBF0FBECDBFC5
:101A6000DF91CF911F910F91FF90EF90DF90CF907A
:101A7000BF90AF909F9008951F93CF93DF93CDB702
:101A8000DEB72C970FB6F894DEBF0FBECDBF4F83E5
:101A9000588769877A878B879C87CE0107960E9433
:101AA0006C0B8823D1F09F8188852A853B85232B69
:101AB00031F08F3F31F481E09F3F19F403C081E0A2
:101AC00001C080E080FD47C04F81588569857A85D7
:101AD0008B859C850E94DE083EC086E0FE0137961D
:101AE000DE01119601900D928A95E1F7FF81E8855C
:101AF0006A857B856115710531F0EF3F31F481E036
:101B0000FF3F19F403C081E001C080E080FD23C0E5
:101B10002091020230E0C901019687709927409117
:101B2000010250E084179507F1F1F983EA837D8380
:101B30006C8396E0929FD001939FB00D1124AD5F0E
:101B4000BD4FFE01319601900D929A95E1F7809379
:101B500002020E94C50A16E08091010290910202E1
:101B6000891771F1189FC00111248D5F9D4F0E944C
:101B70006C0B882329F1E09101021E9FF0011124D2
:101B8000ED5FFD4F40815181628173818481958138
:101B90000E94DE088091010290E0019687709927EB
:101BA00080930102D9CF0E94A808109202021092DD
:101BB0000102E3E3F2E086E0DF011D928A95E9F796
:101BC0002C960FB6F894DEBF0FBECDBFDF91CF913C
:101BD0001F91089580915902859585958595089561
:101BE000809159028770089590915902977081E011
:101BF00009F480E0089580917C02089590917C0220
:101C0000892B80937C020895809590917C02892392
:101C100080937C02089510927C02089590917B023B
:101C2000892B80937B020895809590917B02892374
:101C300080937B02089510927B02089580915A024E
:101C4000089508950C94210E0C94220E9091E702B1
:101C500092FD08C090915A02981721F080935A0281
:101C60000C94240E089580915A02882329F0109232
:101C70005A0280E00C94240E0895CF93DF93E091F4
:101C80000201F091030180917C028083E0910201C6
:101C9000F0910301908180917B02892B8083809158
:101CA0005A02882381F0E0910201F09103019081B2
:101CB000892B808380910201909103010E94DB2493
:101CC00081110E94330EC0910201D091030140E2C4
:101CD00050E069E372E0CE010E943F2E892B69F04B
:101CE00080E2FE01A9E3B2E001900D928A95E1F74E
:101CF000CE01DF91CF910C948724DF91CF9108958D
:101D00000C94210E9091E70292FD10C098E0899FFB
:101D100090011124262B209359020E946009809182
:101D200059028595859585950C94800E0C946009D3
:101D30001092590280E00C94800E209159028095F7
:101D4000822380935902982F977099F430E0482F9E
:101D5000082E000C550B2417350759F09091E70217
:101D600092FD07C08595859585950E9481090C9403
:101D7000980E08959091E70292FB222720F92817E8
:101D800069F080FB92F99093E7028091E6029091CE
:101D9000E7020E94080F82E00C949D0E0895809146
:101DA000E70282FB882780F991E089270C94BA0E1C
:101DB00081E00C94BA0E80E00C94BA0E6FEF7FEFC6
:101DC00080E090E00C947E2E80E090E00E945A2EFD
:101DD00021E0893E9E4F09F020E0822F089582E0A5
:101DE00090E00C944C2E83E090E00C944C2ECF931A
:101DF00084E090E00E944C2EC82F82E290E00E9486
:101E00004C2E2C2F30E0A901582BCA01CF910895F8
:101E1000CF93C92F682F84E090E00E94602E6C2F32
:101E200082E290E0CF910C94602EAB01BC018FE078
:101E300090E00C94722EAB01BC0183E190E00C9415
:101E4000722E60E070E0CB010C941B0F60E070E03C
:101E5000CB010E94150F0C94210F69EE7EEF80E0FC
:101E600090E00E947E2E60E082E090E00E94602E72
:101E700060E083E090E00E94602E1092FD011092DD
:101E8000FE011092FF011092000260E084E090E0F9
:101E90000E94602E60E082E290E00E94602E60E08E
:101EA00085E090E00E94602E60E086E090E00E9475
:101EB000602E6FEF87E090E00E94602E40E050E0DF
:101EC000BA0188E090E00E94722E60E08DE090E020
:101ED0000E94602E40E050E0BA0188E190E00E944C
:101EE000722E60E087E190E00E94602E40E050E0BA
:101EF000BA018CE190E00E94722E60E070E080E216
:101F000090E00E947E2E40E050E0BA0188E190E02F
:101F10000E94722E0C94260F0C942D0F682F8EE0C9
:101F200090E00C94602E0E94412660938B02709387
:101F30008C0280938D0290938E026093870270933F
:101F400088028093890290938A02089585B78068F9
:101F500085BF85B7806885BF089581E008950C949A
:101F6000AD0F08950C94B10F0C94B10F0C94B40FF5
:101F70000C94B10F0C94B80F0C94B10F0E94A60FE3
:101F800084E892E10E9471240E94BC0F0C94BA0F65
:101F90000E94B20F0C94B10F0E949E120E94620424
:101FA0000C94A2200E942C260E9483130E94CC0F26
:101FB0000E94401E0E94411C0C94B60F5F926F92CB
:101FC0007F928F929F92AF92BF92CF92DF92EF92C9
:101FD000FF920F931F93CF93DF93CDB7DEB72A976E
:101FE0000FB6F894DEBF0FBECDBF0E949813C82E67
:101FF00081110E94930F3DE7832E32E0932E00E083
:1020000010E0502E802F0E94C2125C01F4016190FA
:1020100071904F016826792661147104B1F40F5F45
:102020001F4F0530110569F78FEF89838A831B8263
:102030000E9435268160782F9D838C8349815A8147
:102040006B818D810E947E043AC080918F0281FD58
:102050000E94CB12D12CEE24E394F12CC3018E21EB
:102060009F21892B29F10E94AF0F8823A9F0DE82DE
:102070005F82AE20BF2081E0AB2809F480E0888732
:102080000E9435268160782F9A8789874E815F81EB
:1020900068858A850E947E04000F111FF801E358AD
:1020A000FD4F80819181E826F926F182E08207C008
:1020B000D394EE0CFF1CFEE0DF12D0CFB0CF81E056
:1020C000C11001C080E02A960FB6F894DEBF0FBEA3
:1020D000CDBFDF91CF911F910F91FF90EF90DF90D7
:1020E000CF90BF90AF909F908F907F906F905F90B8
:1020F00008950E94DE0F0E94851C0E9406200E9407
:102100009F150C947304CF93DF930E94AD11EC01E3
:10211000811521E5920708F045C0811530E5930748
:1021200008F094C0883E910528F5803E910508F09E
:10213000F8C0883A910570F4853A910508F07CC0A2
:102140008130910509F475C008F4E8C0049708F0DF
:10215000E8C0E4C08F3B910508F0E0C0C85AD0E069
:10216000CC0FDD1FC15ADE4F0990D881C02DCE01A2
:102170009464D8C0811540E2940758F4811551E069
:10218000950708F0CEC08D3E910508F4C7C0906554
:10219000C9C0C11580E4D80708F4C0C0DF70CE0103
:1021A000906AC0C0811525E59207A8F4811534E531
:1021B000930708F095C0811543E5940708F07BC0AC
:1021C000811552E5950708F061C0D82FCC27CE01C4
:1021D000816F906AA7C0C11589E5D807A0F4C11521
:1021E00028E5D20708F082C0C11536E5D30708F00C
:1021F00095C08C2F0E9441128F7190E0D82FCC2770
:10220000CE0190628FC0C1154AE5D40708F474C0AE
:10221000CE0190568115904208F080C08D2F8F71AD
:102220000E944112DD27D0628F71AE01582BCA0186
:1022300079C081E090E076C0C55AD0E0C357DE4F48
:102240008881C82FD0E0CE0190646CC074E0969570
:1022500087957A95E1F7282F23703C2F337081E022
:1022600090E002C0880F991F3A95E2F79C68AC0194
:10227000522B9A019C2F9F709695969550E2959FB0
:10228000E0011124C9018C2B9D2B4CC08370992730
:1022900021E030E002C0220F331F8A95E2F79C2F25
:1022A0009695969580E2989FE0011124C22BD32B3E
:1022B000CE019C6837C08370992721E030E002C0CE
:1022C000220F331F8A95E2F79C2F9695969540E250
:1022D000949FE0011124C22BD32BCE019A6822C017
:1022E000D82FCC27CE01846F906A1CC0DC2FCC275E
:1022F000CE01806F906A16C08C2F8F700E944112A1
:1023000094E0D695C7959A95E1F7CF70D0E0DC2F91
:10231000CC27D0699E01282BC90104C080E090E041
:1023200001C0CE01DF91CF91089526E4829FC001C4
:102330001124FC012EE0729FE00DF11D1124E60F27
:10234000F11DEE0FFF1FEC59FE4F859194910895FA
:102350000E9495110E94831008958238910569F1B9
:10236000B0F48133910509F46DC048F489329105C8
:1023700009F463C08A32910509F469C00895853370
:10238000910509F455C089339105B9F00895833E4C
:10239000910569F138F4803E9105B1F0823E9105D6
:1023A00009F10895863E9105A9F1873E9105B9F19D
:1023B000843E910509F064C023C02091E60220FD0F
:1023C0004FC021FD4DC008958091E60280FD44C0BC
:1023D0008091E70280FF44C08091E60284FD42C004
:1023E00083EE4DC08091E60282FF38C0F5CF809128
:1023F000E60282FD33C08091E70280FD31C0ECCF60
:102400008091E70281FF32C08091E60284FD2AC0FC
:1024100087EE35C08091E60283FF26C0F5CF80911C
:10242000E60283FD21C08091E70281FD1FC0ECCF51
:102430008091E60285FD1CC01DC08091E60285FDED
:1024400019C016C08091E60286FD16C017C08091A3
:10245000E60286FD13C010C089E311C082EE0FC0F2
:1024600080EE0DC080E00BC086EE09C084EE07C090
:1024700089E205C085E303C08AE201C081E390E000
:1024800008959091E60292FF0DC0282F2871283000
:1024900019F4877F846006C0282F2471243011F43A
:1024A0008B7F886093FF0DC0282F2871283119F485
:1024B000877E846106C0282F2471243111F48B7E1D
:1024C00088612091E70220FF0DC0382F3871383025
:1024D00019F4877F816006C0382F3171313011F4D3
:1024E0008E7F886021FF0DC0282F2871283119F4B4
:1024F000877E816106C0282F2171213111F48E7EE3
:10250000886194FD877E089580E008950C94DE0E26
:102510000E9498138FE39CE90197F1F700C0000037
:102520000E94981380E00E94C21280FF04C00E94A3
:1025300086120C94822608950C9488120E94E40E50
:10254000811102C00E948C0F0E94EF0E80938F02B7
:102550000E94F70E9093E7028093E6020E949C127D
:102560000E94F30E682F70E080E090E00E94000966
:102570006091F9017091FA018091FB019091FC0149
:102580000C943809E82FF0E0EE0FFF1FEE50FD4FDE
:10259000808191810895089580EA8A95F1F70895E0
:1025A00000C008950C94CC1208950C94D4120C948D
:1025B000D5120C94D4120C94D912F894E82FE29509
:1025C000EF70F0E031A1282F2F7081E090E001C082
:1025D000880F2A95EAF7982F9095932391A392A1BB
:1025E000892B82A3789408950F931F93CF93DF9341
:1025F000CEE9D1E089918F3F11F00E94DD1281E098
:10260000C33AD807B9F7C0E9D1E00EE911E08991E2
:102610008F3F11F00E94DD120C171D07C1F7DF91EB
:10262000CF911F910F910895BF92CF92DF92EF92B9
:10263000FF920F931F93CF93DF938C01C62FD0E0AF
:10264000CE0182569E4F6C01FC0190819F3F09F4A0
:1026500050C0B62EF894E92FE295EF70F0E081A11A
:102660009F7021E030E001C0220F9A95EAF7822B9B
:1026700081A382A12095282322A378940E94D012BE
:10268000E0E9F1E04EE951E021E030E0E12CF12C0D
:1026900061916F3F89F0A62FA295AF70B0E0909640
:1026A0008C9190E06F7002C0959587956A95E2F7DE
:1026B00080FD02C0C90102C080E090E0E82AF92A4A
:1026C000220F331F4E175F0719F7F60180818F3FE6
:1026D00011F00E94DD1261E0E114F10409F460E000
:1026E0008B2D0E94D212CC0FDD1FC00FD11FF9829B
:1026F000E882DF91CF911F910F91FF90EF90DF90D3
:10270000CF90BF9008950E94F4128AE0E2EFF2E0C9
:10271000DF01982F1D929A95E9F7E8EEF2E0DF01CC
:102720001D928A95E9F785E00E94E3130C94D60385
:10273000FF920F931F93CF93DF93CDB7DEB72A9706
:102740000FB6F894DEBF0FBECDBF8E010F5F1F4FD7
:102750008AE0F80111928A95E9F7F12C6F2DC801F2
:102760000E941413F394F5E0FF12F8CF4AE050E012
:10277000B80188EE92E00E943F2EFF24F394009768
:1027800009F4F12C892B41F08AE0F801A8EEB2E0BF
:1027900001900D928A95E1F72F2D45E062EF72E0EE
:1027A00088EE92E00E94E4130E94D8038F2D2A96AF
:1027B0000FB6F894DEBF0FBECDBFDF91CF911F9152
:1027C0000F91FF9008950895FF920F931F93CF9359
:1027D000DF93F82E092F162FD72FC42F222349F06D
:1027E00081E0809392020E9435269093910280931B
:1027F0009002809192028823D9F08091900290916A
:1028000091020E944D26059798F0EF2DF02FA12FF1
:10281000BD2F80E090E04C2F50E08417950734F4F2
:10282000219131912D933D930196F7CF1092920211
:10283000DF91CF911F910F91FF9008950E944D2835
:102840000E94D20F0C9459280E945D280E94791092
:102850000C9477280E94D3250E9434280E94BE0F32
:102860000E941E140E9424140E94C80FFBCF809166
:10287000990280FF06C06091090170E0660F771F22
:1028800026C081FF04C06091090184E005C082FF79
:1028900007C06091090188E0689FB001112417C04A
:1028A000909198029923D1F060910801961788F7CA
:1028B0002091090188E0289F90011124929FA00196
:1028C000939F500D112470E0CA010E94B92D603809
:1028D000710540F46115710519F406C068E070E0F7
:1028E000862F08958FE7089581E0089580919902D9
:1028F00080FF08C06091050170E07595679575953A
:10290000679521C081FF06C06091050170E0759553
:10291000679519C082FF04C06091050170E010C086
:1029200090919702992399F0609104019617A0F76E
:1029300080910501899FC001112470E00E94B92D8A
:102940006038710540F46115710519F406C061E045
:1029500070E0862F08958FE7089581E008958D3EF9
:1029600021F40E943714819504C08E3E29F40E9400
:10297000371480939D0208958F3E21F40E943714EE
:10298000819504C0803F29F40E94371480939C02F3
:102990000895893F19F40E94761405C08A3F31F4E6
:1029A0000E947614819580939E0208958B3F21F4B6
:1029B0000E947614819504C08C3F29F40E947614FD
:1029C00080939F0208959FE0980F983078F421E05B
:1029D00030E0A90102C0440F551F9A95E2F7CA01E1
:1029E00090919B02892B80939B0208958D3F21F447
:1029F0008091990281600BC08E3F21F480919902F1
:102A0000826005C08F3F29F4809199028460809391
:102A1000990208958D3E39F490919D0297FF35C03B
:102A200010929D0259C08E3E29F490919D02191674
:102A3000BCF32BC090919C028F3E29F497FF25C0D8
:102A400010929C0249C0803F19F41916CCF31DC0A6
:102A500090919E02893F29F41916BCF410929E02AF
:102A60003BC08A3F19F497FF10C0F8CF8B3F39F471
:102A700090919F0297FF09C010929F022DC08C3F3A
:102A800021F490919F021916BCF39FE0980F9830A3
:102A900080F421E030E0A90102C0440F551F9A954F
:102AA000E2F7CA01809590919B02892380939B0253
:102AB00013C08D3F21F4809199028E7F0BC08E3F11
:102AC00021F4809199028D7F05C08F3F29F4809178
:102AD00099028B7F8093990280919C02811106C09C
:102AE00080919D02811102C01092980280919E02F5
:102AF000811106C080919F02811102C0109297023D
:102B000008950E94352620919C02211104C0209135
:102B10009D02222321F090939602809395022091AA
:102B20009E02211104C020919F02222321F0909344
:102B30009402809393028AE992E00C94A124EF928C
:102B4000FF920F931F93CF93DF9300D000D000D05C
:102B5000CDB7DEB786E0EAE9F2E0DE01119601903A
:102B60000D928A95E1F7E0909C02F0909D02009111
:102B70009E0210919F0210929C0210929D02109250
:102B80009E0210929F02E11003C0FF2009F45DC075
:102B900080919502909196020E944D26AC019091F1
:102BA0009802992339F020910A0130E02417350763
:102BB00058F04BC020910B018AE0289F900111240E
:102BC0002417350718F041C09F3F19F09F5F90937D
:102BD0009802EE2061F00E9437141E1414F09FEF4B
:102BE00001C091E0989F902D112490939C02FF20AA
:102BF00061F00E9437141F1414F09FEF01C091E0A0
:102C0000989F902D112490939D0230919C02332324
:102C1000E1F020919D022223C1F045EB3403C00175
:102C20001124992319F090939C0203C081E08093B2
:102C30009C0235EB2303C0011124992319F09093D2
:102C40009D0203C081E080939D02011103C0112306
:102C500009F45DC080919302909194020E944D26E8
:102C6000AC0190919702992339F02091060130E050
:102C70002417350758F04BC0209107018AE0289FA0
:102C8000900111242417350718F041C09F3F19F017
:102C90009F5F90939702002361F00E9476141016B4
:102CA00014F09FEF01C091E0989F902D1124909314
:102CB0009E02112361F00E947614111614F09FEF0A
:102CC00001C091E0989F902D112490939F02309124
:102CD0009E023323E1F020919F022223C1F045EBB5
:102CE0003403C0011124992319F090939E0203C06C
:102CF00081E080939E0235EB2303C00111249923C8
:102D000019F090939F0203C081E080939F0280910D
:102D10009C0281110BC080919D02811107C080919E
:102D20009E02811103C080919F0281110E94811532
:102D3000EB82FC820D831E8386E0FE013196AAE9B8
:102D4000B2E001900D928A95E1F726960FB6F894BD
:102D5000DEBF0FBECDBFDF91CF911F910F91FF90CE
:102D6000EF900895EAE9F2E086E0DF011D928A958E
:102D7000E9F7109298021092970210929902089522
:102D8000EF92FF920F931F93CF93DF938B01682FE6
:102D900011110AC0442329F0E82FF0E0ED5EFB4F4B
:102DA0006491762F862F75C0212F30E0E82FF0E058
:102DB000442321F0ED5EFB4FE491F0E046E0049FF8
:102DC000C0011124CFEFD0E0BE010E94A52D4BEA37
:102DD0004603C001479F900D1124800F911D800F65
:102DE000911D982F990F890FAE01421B530B4E9FD7
:102DF000D0014F9FB00D5E9FB00D11249B2F189FE7
:102E0000A0011124452F55278E01041B150B0E9F81
:102E1000A0010F9F500D1E9F500D11247E01E81A36
:102E2000F108E29E8001E39E100DF29E100D112428
:102E3000212F3327C21BD30BCE9F9001CF9F300D84
:102E4000DE9F300D112462307105A9F048F4611540
:102E5000710569F061307105C9F48B2F752F0DC0B4
:102E60006430710581F058F06630710579F47E2F79
:102E70008B2F932F0DC0832F7B2F9E2F09C08E2F5A
:102E80007B2F952F05C08E2F732F02C07E2F852F8D
:102E9000692FDF91CF911F910F91FF90EF900895CF
:102EA00041E00E94C016089508950E9450170895A9
:102EB000CF93DF93762FE901682F842F0E94551757
:102EC000798368838A83DF91CF910895493C08F024
:102ED00048EC0C9458178091FC02282F269530E07E
:102EE0002115310519F48170826005C02532310544
:102EF00024F0817088648093FC028091FF02893CF9
:102F000018F088EC8093FF02089588E090E00C941C
:102F1000542ECF92DF92EF92FF926B017C010E94C0
:102F20006B17B701A60188E090E0FF90EF90DF906B
:102F3000CF900C94722EECEFF2E083E0808311824C
:102F40008FEF828388EC8383148260817181828118
:102F500093810C9489178091FC0280FF02C08695B2
:102F6000089580E0089590910003933018F49F5FD6
:102F700090930003882351F06091FC027091FD0250
:102F80008091FE029091FF020C948917089581E0D0
:102F90000C94B31790910003992319F091509093DA
:102FA0000003882351F06091FC027091FD02809132
:102FB000FE029091FF020C948917089581E00C9411
:102FC000CA1770E00C94B820609110018091FC0247
:102FD00080FF0AC080910F0123E0829FC00111246D
:102FE0008F5F9C4F0C94E117809111019091120119
:102FF000891780F7E82FF0E09F01220F331FE20FBF
:10300000F31FEF5FFC4F1182108212828F5FF0CFAF
:103010009091FC0290FF16C0909111012091120135
:10302000921770F4E92FF0E0DF01AA0FBB1FEA0F3F
:10303000FB1FEF5FFC4F8183608342839F5FF0CF74
:103040000C94E4170895CF93DF9300D01F92CDB76F
:10305000DEB79091FC0290FF0AC09E012F5F3F4FA8
:103060000E9466174B8169818A810E9408180F901F
:103070000F900F90DF91CF910895CF93DF93EC01E4
:10308000EC81F0E0E257FD4F4491ECEFF2E0628119
:1030900081810E9423188C818F5F8C83DF91CF9177
:1030A0000895CF93DF93EC01ECEFF2E0438162816E
:1030B0008C810E9423188C818F5F8C83DF91CF914C
:1030C00008950F931F93CF93DF9300D01F92CDB736
:1030D000DEB78C018091A00281110AC09E012F5F92
:1030E0003F4F48EC6FEF0E9466178A818093A002E1
:1030F000F8018481813051F028F0823061F44091F0
:10310000A0020AC08091A00240E007C06091A00226
:1031100040E080E003C040E080E060E00E940818EA
:10312000F801848190E0019663E070E00E94B92D7F
:1031300084830F900F900F90DF91CF911F910F918B
:103140000895AF92BF92CF92DF92EF92FF920F93CA
:103150001F93CF93DF9300D01F92CDB7DEB7182F08
:10316000F62E042FE22E9091FC0290FF6DC0E92F05
:10317000E695AE2FB0E0AD55BE4F8C918093AC027A
:103180009E7F923061F49E012F5F3F4F812F0E94FE
:1031900066174B8169818A810E94081843C082307A
:1031A00019F40091FF023EC0863019F41091FD021F
:1031B00039C08930D9F38931A9F5E9518E2F817051
:1031C000D82EE695F0E0E257FC4FA590B490C12CC4
:1031D000BB2460911301C61618F52C2D30E0A29E79
:1031E000C001A39E900DB29E900D112470E00E942C
:1031F000A52D812FD11002C0860F01C0861B909192
:103200001101290F311DA901440F551F240F351F2E
:103210002F5F3C4F402F6F2D0E946617C394D9CF6C
:103220000E94E4171093FD02F092FE020093FF0249
:10323000EE2051F06091FC027091FD028091FE023F
:103240009091FF020E9489170F900F900F90DF91CD
:10325000CF911F910F91FF90EF90DF90CF90BF9093
:10326000AF900895ECEFF2E09181282F43816281C5
:1032700088E0890F0C94A11881E00C943219ECEFCE
:10328000F2E09181282F4381628188EF890F0C94AD
:10329000A11881E00C943F19ECEFF2E0628128E084
:1032A000620F08F46FEF282F438181810C94A118DD
:1032B00081E00C944C19ECEFF2E0628128E0621B93
:1032C00008F460E0282F438181810C94A11881E0EB
:1032D0000C945B19ECEFF2E0438128E0420F08F414
:1032E0004FEF282F628181810C94A11881E00C940A
:1032F0006A19ECEFF2E0438128E0421B08F440E059
:10330000282F628181810C94A11881E00C94791995
:1033100020E00C94A118FF920F931F93CF93DF939B
:10332000EC01F12C0FEF10E060911301F616F0F4B0
:10333000809111012F2D30E0280F311DC901880F18
:10334000991F280F391F2F5F3C4F70E0C8010E9462
:10335000B92D962F8C814091FF026091FE02F99E5B
:10336000800D11240E946617F394DECF0E94E417AB
:103370009A818C8190FF02C08F5F01C081508C8345
:10338000DF91CF911F910F91FF900895AF92BF925F
:10339000CF92DF92EF92FF920F931F93CF93DF9321
:1033A000FC01828180FF02C00FEF01C001E010E04C
:1033B0004EE0A42E80911301181708F043C08091AD
:1033C0001101C12ED12CE601C80FD11DCE01880FED
:1033D000991FC80FD91FCF5FDC4F198218821A823C
:1033E00034E0E32EF12CB12C8091A2028B0D8F30B2
:1033F0002CF06A2D0E94972D892F05C087FF03C0EE
:1034000090911301890F082E000C990BC816D9064C
:1034100091F48091FF028E9DA0018F9D500D11248B
:1034200055954795559547959E016091FE0280916F
:10343000FD020E946617B00EF1E0EF1AF108A1F646
:103440001F5FB8CF0E94E4178091A202013031F4CF
:10345000811102C080911301815007C090E0019654
:103460006091130170E00E94B92D8093A202DF9158
:10347000CF911F910F91FF90EF90DF90CF90BF9071
:10348000AF900895CF938091110190911201891707
:1034900070F4E82FF0E09F01220F331FE20FF31FBB
:1034A000EF5FFC4F1182108212828F5FF0CFC0E07D
:1034B00060911301C617C0F5EC2FF0E070E0CF016A
:1034C0000E94B92D20911101820F2091A102022E9C
:1034D000000C330B90E0E217F307CCF020910E01C3
:1034E000022E000C330B2E173F078CF09C01220F8D
:1034F000331F820F931F9C012F5F3C4F4091FF02AF
:103500006091FE028091FD020E9466170BC0FC01D3
:10351000EE0FFF1F8E0F9F1FFC01EF5FFC4F11820C
:1035200010821282CF5FC4CF0E94E41720910D0158
:103530008091A102820F8093A10290910E01920FBF
:1035400090930E0119165CF4082E000C990B409113
:10355000130150E041505109841795071CF0219543
:1035600020930D01CF9108958F929F92AF92BF92B9
:10357000CF92DF92EF92FF920F931F93CF93DF933F
:103580008C01FC014481C42FD0E09E01DE010E9429
:10359000FD2D9B01AC010E94132E6B017C01E0E22A
:1035A000F0E0EC1BFD0BA5E5B0E09B01AC010E9437
:1035B000132E4B015C019F01DF010E94F52D9B0141
:1035C000AC010E941E2E9B01AC012C0D3D1D4E1D19
:1035D0005F1DC501B4010E94CD2DC22FD22F2A320A
:1035E00028F4F3E02F9F900111240DC025E530E071
:1035F0002C1B3109C901880F991F280F391F37FF6C
:1036000002C02F5F3F4F35952795C22FC095F12CF3
:1036100085E5E82EED1A80911301F816C8F4F1FC47
:1036200002C08E2D01C08D2F909111012F2D30E001
:10363000290F311DA901440F551F240F351F2F5F7E
:103640003C4F4C2F6091FE020E946617F394E3CF2B
:103650000E94E417F8018481811102C091E003C047
:10366000803219F49FEF90930C0190910C01890F17
:10367000F8018483DF91CF911F910F91FF90EF901C
:10368000DF90CF90BF90AF909F908F9008950F9351
:103690001F93CF93DF93EC0100E010E080911301C2
:1036A000282F30E00217130724F59091110198019B
:1036B000290F311DA901440F551F240F351F2F5FFE
:1036C0003C4F869590E04C81081719071CF4442361
:1036D00031F002C0411103C04091FF0201C040E03F
:1036E0006091FE028091FD020E9466170F5F1F4FDE
:1036F000D5CF0E94E4178C8190E0019681709927C4
:103700008C83DF91CF911F910F910895ECEFF2E040
:1037100080818E7F808360817181828193810E940C
:1037200089171092AD022FEF80E792E02150804080
:103730009040E1F700C000000C94E417ECEFF2E0D9
:1037400080818E7F80831092AD022FEF80E792E020
:10375000215080409040E1F700C000000C94E41735
:103760001092AD028091AA0281110AC081E080937B
:10377000AA028091FC0281708093A9020C949E1B86
:1037800008956091FC02669570E04BE050E084E1A2
:1037900091E00E94322E892B19F481E08093AD02D2
:1037A0000E9435269093A4028093A30208959091DD
:1037B000FC0290FF35C09170811102C0926006C07A
:1037C000853210F0986402C0880F982B9093FC0209
:1037D000662351F06091FC027091FD028091FE021F
:1037E0009091FF020E9489176091FC02669570E03B
:1037F0004BE050E084E191E00E94322E892B19F0D9
:103800001092AD0202C00E94C11B81E08093A6020B
:103810004091FF026091FE028091FD020C94881994
:103820000895682F9091FC02969581E0890F85326A
:1038300008F081E00C94D71B81E00C94111C682FD8
:103840009091FC0296958FEF890F09F484E20C9415
:10385000D71B81E00C941F1C61E00C94D71BECEF8C
:10386000F2E080818160808386950C942C1C80918D
:10387000FC0280FD0C94861B0C942F1C60E00C94C1
:10388000D71B8091AB0281112EC00E94E40E8111E2
:1038900004C00E948C0F0E949B170E9485176093A2
:1038A000FC027093FD028093FE029093FF026E7FF4
:1038B00061F40E949B170E9485176093FC0270932D
:1038C000FD028093FE029093FF020E946B171092FC
:1038D000AD028091FC0280FF03C086950E943E1CD1
:1038E00081E08093AB020895ECEFF2E0808181608B
:1038F000808386950C943E1C1092AA028091A902A6
:1039000081110E94741C0C94C11B0F931F93CF93C1
:10391000DF938091AD02882309F485C08091AC02C9
:10392000E091FC02E695E81BE093A502823049F4A1
:10393000F0E0E657FD4FE491CE2FD0E00DE318E123
:1039400049C0863049F4F0E0E957FD4FE491CE2FAD
:10395000D0E001E518E13EC0893051F4E695F0E091
:10396000EC57FD4FE491CE2FD0E00BE819E132C0C7
:103970008F3051F4E695F0E0EF57FD4FE491CE2FF4
:10398000D0E006EC19E126C0853149F4F0E0E258B8
:10399000FD4FE491CE2FD0E002E41AE11BC0883144
:1039A00081F0833239F4ECE7F2E0C591D49101E67D
:1039B00018E110C0843251F4C4EFD1E007E41BE1F8
:1039C00009C0C8E2D0E004EB1AE104C0C0EDD7E0C2
:1039D00004E517E18091A602882361F01092A60207
:1039E0000E9435269093A4028093A3021092A8020D
:1039F0001092A7020E943526E091A302F091A40242
:103A00008E1B9F0B8F3F9F4770F4EC0FFD1FF093B1
:103A1000A402E093A30283EA92E0F801DF91CF9140
:103A20001F910F910994DF91CF911F910F910895EC
:103A3000882311F0FA0101C0FB010994CF93DF93B1
:103A4000C82FD62F0E94AB178C1740F00E94AB17DF
:103A50008D1720F4DF91CF910C941C1C8C2FDF91DB
:103A6000CF910C942C1C1F93CF93DF93FB011281F9
:103A70001111C3C0EC010E94FB0D8272CD3CFCE52C
:103A8000DF0709F49AC0A8F5C73CECE5DE0709F4A6
:103A900076C0A8F4C43C9CE5D90709F45FC028F4BB
:103AA000C33CDC4509F457C054C0C53C9CE5D9076C
:103AB00009F459C0C63CDC4509F45CC04AC0CA3CA4
:103AC000FCE5DF0709F46AC050F4C83CECE5DE070A
:103AD00009F45AC0C93CDC4509F45BC03AC0CB3C90
:103AE0009CE5D90709F45FC0CC3CDC4509F460C013
:103AF00030C0C23DFCE5DF0709F46FC088F4CF3C5D
:103B00009CE5D90709F460C008F45CC0C03DFCE541
:103B1000DF0709F45CC0C13DDC4509F45BC019C096
:103B2000C53D9CE5D90709F460C050F4C33DFCE5F0
:103B3000DF0709F455C0C43DDC4509F454C009C091
:103B4000C63D9CE5D90709F455C0CE35DD4509F4DD
:103B500054C011E052C00E94371C4FC049E25CE1E2
:103B60006CE17CE104C04CE15CE169E27CE10E9433
:103B7000181D43C049E459E16CE379E1F8CF4CE307
:103B800059E169E479E1F3CF47E659E168E579E184
:103B9000EECF48E559E167E679E1E9CF45E859E13B
:103BA00066E779E1E4CF46E759E165E879E1DFCFFF
:103BB0004EED57E167EC77E1DACF47EC57E16EED78
:103BC00077E1D5CF81E017C065E082E010C068E002
:103BD00086E00DC06EE089E00AC064E18FE007C0B6
:103BE00067E185E104C088E106C062E289E10E94E4
:103BF0001E1D03C083E20E942C1C812FDF91CF91F8
:103C00001F91089586E090E00C944C2E682F86E07A
:103C100090E00C94602E80912B03847089628093D5
:103C20002B030C94061E80912B0386958695869512
:103C3000089580912B0381FD07C0826080932B0340
:103C40000E94061E0C940720089580912B0381FF8B
:103C500007C08D7F80932B030E94061E0C941320B7
:103C6000089580912B0381FD0C94251E0C94191E40
:103C700080912B0386958170089580911F0108958E
:103C80000E94E40E811104C00E948C0F0E940B1E42
:103C90000E94021E80932B03282F26952695269599
:103CA00030E02630310524F08770886280932B0342
:103CB00080912B0380FF04C086958695869501C070
:103CC00080E00C94D41F20912B03822F869586953B
:103CD0008695482F50E04530510554F48F5F982F5A
:103CE000990F990F990F822F8770892B80932B033F
:103CF00080912B03816080932B030E94061E80918C
:103D00002B038695869586950C94D41F80912B0362
:103D1000982F969596959695A1F0915E990F990F8B
:103D2000990F8770892B80932B03887F91E009F48A
:103D300090E080912B0390FB80F980932B030E94ED
:103D4000061E80912B038695869586950C94D41F2C
:103D500080912B0380FD13C0816080932B03813001
:103D600019F489E080932B0380912B030E94061E97
:103D700080912B038695869586950C94D41F089583
:103D800080912B0380FF08C08E7F80932B030E94BD
:103D9000061E80E00C94D41F089580912B0380FDB3
:103DA0000C94C01E0C94A81E90912B03892F86950D
:103DB000869586958F5F8F719770863038F4880F5F
:103DC000880F880F892B80932B0302C090932B03BD
:103DD00080912B03887F91E009F490E080912B0380
:103DE00090FB80F980932B030E94061E80912B0389
:103DF0008695869586950C94D41F863008F085E0CC
:103E000090912B039770282F220F220F220F922BB5
:103E100090932B03987F21E009F420E090912B03ED
:103E200020FB90F990932B030C94D41F0E94FD1E4D
:103E300080912B030C94061EFC01DB0112968C91E1
:103E40008823F9F0EC5BFC45E730F105D8F4EE5936
:103E5000FF4F0C94EF2D85E001C080E00E94161FFB
:103E600080E008950E94861EFBCF0E94631EF8CF5B
:103E70000E94CD1EF5CF0E94D41EF2CF0E94311EAB
:103E8000EFCF81E00895279A2F9808952F980895ED
:103E90008F929F92AF92BF92CF92DF92EF92FF925A
:103EA0000F931F93CF93DF938C01809186009091A5
:103EB00087006CE070E00E94A52D6017710730F05C
:103EC000C80169E070E00E94A52D60C08091860065
:103ED00090918700E0908600F0908700E091860046
:103EE000F0918700C6E0D0E0BE010E94A52D20E041
:103EF00030E0060F171F211D311D4801590185E0D3
:103F0000880C991CAA1CBB1C8A95D1F7C701BE015D
:103F10000E94A52D6F01E12CF12CA7019601260F1F
:103F2000371F411D511DC501B4010E94CD2D6901EE
:103F30007A01E0918600F0918700CA01B9010E94E0
:103F4000872D9B01AC01DF010E94132E9B01AC0168
:103F5000C701B6010E94872DDC01CB012FE0B69589
:103F6000A795979587952A95D1F70091860010918E
:103F7000870020E030E0081719072A073B0728F4DC
:103F80006091860070918700CB01BC01CB01DF916D
:103F9000CF911F910F91FF90EF90DF90CF90BF9046
:103FA000AF909F908F900895CF93C82F863050F494
:103FB000811109C080918000877F809380000E94DA
:103FC000461F06C0C5E08091800088608093800015
:103FD000A0918600B09187002C2F30E00E94FD2D2B
:103FE00025E030E040E050E00E94CD2DB42FA32F1B
:103FF000922F8827892F9A2FAB2FBB270E94481F0B
:1040000090938D0080938C00CF9108950895109225
:10401000AF021092AE021092B002EFE6F0E08081A3
:10402000816080830895EFE6F0E080818E7F808359
:104030000E94131E0C94D41F1F920F920FB60F9262
:1040400011240F931F932F933F934F935F936F937D
:104050007F938F939F93AF93BF93CF93EF93FF93F0
:104060008091200191E0980F823019F09093200107
:1040700055C081E0809320010E943D1EC82F009111
:10408000AE021091AF020F5F1F4F0E943D1E28E746
:10409000829FB0011124C8010E94A52D9093AF0208
:1040A0008093AE0228E7C29FB0011124660F672FEC
:1040B000661F770B71950E94A52D6F778091B002D6
:1040C000823019F4603451F404C0813039F46F3710
:1040D00029F480916F008E7F80936F00E62FF0E0CF
:1040E000ED56FC4FC49100918600109187000E940C
:1040F000131E282FC09FC001C19F900D11246BEF8C
:1041000074E00E94A52D269FC001279F900D1124C9
:104110000E94481F90938D0080938C00FF91EF9137
:10412000CF91BF91AF919F918F917F916F915F914F
:104130004F913F912F911F910F910F900FBE0F90B4
:104140001F9018950E94431F8AE08093800089E1A8
:10415000809381008FEF9FEF90938700809386007C
:104160000E94401E0E94381E81110C940720089561
:10417000529A2BB12B7F3BB134604FB7F894FC01BE
:10418000CB01880F991F680F791F6E0F7F1FE617ED
:10419000F70789F0819198E03BB9000000C087FFE4
:1041A0002BB9880F000000C000C000C02BB900C0B0
:1041B0009A9591F7ECCF4FBF8FE594E00197F1F717
:1041C00000C000000895CF93DF93EC01FB018281D2
:1041D000882309F43CC1C430FDE5DF0760F4CB3F20
:1041E0009CE5D90788F49E0122503C4524313105D5
:1041F00008F02EC109C0C236EDE5DE0729F0C63A47
:10420000FDE5DF0709F024C10E94F70E9093E70255
:104210008093E602C1318CE5D80709F4C6C008F0E6
:1042200042C0C930ECE5DE0709F49BC000F5C5309B
:104230008CE5D80709F485C078F4C330ECE5DE07D7
:1042400009F478C008F07AC0C230DC4509F0F5C046
:104250008091E6028160EFC0C7309CE5D90709F480
:1042600078C008F07AC08091E6028061E4C0CD3069
:10427000FCE5DF0709F487C058F4CB309CE5D9078B
:1042800009F479C008F07BC08091E60288606FC0B5
:10429000CF30FCE5DF0709F480C008F082C08091D0
:1042A000E602877FC8C0CE3F9CE5D90709F471C0FC
:1042B00000F5C531FCE5DF0709F485C068F4C331BA
:1042C0009CE5D90709F475C008F095C00E94A808BC
:1042D0008091E6028F77AFC0CC3FFCE5DF07A9F104
:1042E00008F054C0CB3FDC4509F0A7C08091E7023D
:1042F00040C0C230EDE5DE0709F489C058F4C115AD
:104300008DE5D80709F45AC008F069C08091E7022A
:1043100082602FC0C236EDE5DE0709F47CC0C63AE4
:10432000FDE5DF0709F481C0C330DD4509F085C034
:1043300080E06EC08091E60282607DC08091E602DE
:1043400016C08091E602886076C08091E7028260A4
:104350004FC08091E60280626EC08091E602806468
:104360006AC00E94A8088091E602806864C08460E8
:1043700062C081603DC08091E6028E7F5CC080910A
:10438000E6028D7F58C08091E60216C08091E70258
:1043900018C08091E7028D7F2BC08091E6028F7E4E
:1043A0004AC08091E6028F7D46C08091E6028F7BF5
:1043B00042C08091E602877F8B7F3DC08091E702FB
:1043C0008D7F8E7F15C08091E60282FB222720F927
:1043D00091E0922790FB82F990FB83F92CC08091A9
:1043E000E702982F909591708E7F892B90FB81F931
:1043F0008093E70222C00E94A8088091E60287FB12
:10440000222720F991E0922790FB87F914C081E0E0
:104410000E948E0F12C08091E60284FB222720F9B1
:1044200091E0922790FB84F906C08091E602982FD4
:10443000909590FB80F98093E6028091E60290913E
:10444000E7020E94080F0E94A80880E001C081E0F6
:10445000DF91CF910895893289F1F0F4843171F1BF
:10446000B0F4873009F077C081E080930B0184E1DC
:1044700080930A018AE0809309018EE1809308010C
:1044800088E08093050188E28093040164C092EE85
:10449000980F9A30F0F05FC0803509F444C028F4DA
:1044A0008F3409F058C08AE03FC0813529F0823549
:1044B00009F051C081E038C08FEF36C08091B3025F
:1044C000882379F11092B3021092B2021092B102D5
:1044D00042C08D518093B302833099F038F481301B
:1044E00069F08230D9F48AE091E00DC0853099F00E
:1044F00078F0863099F484E091E005C08BE091E09B
:1045000002C089E091E09093B2028093B10223C08F
:1045100088E091E0F8CF85E091E0F5CF1092B3020A
:104520001AC080E0089586EFE091B102F091B202E6
:10453000309789F02081082E000C990B820F911D75
:104540008F3F910519F014F08FEF04C097FF02C060
:10455000108201C0808381E008950F931F9341E092
:1045600050E060E070E08A019B0104C0000F111F61
:10457000221F331F8A95D2F7C901B8010E94000992
:104580001F910F910C94A808482F50E0FA0135971D
:10459000EF33F10508F060C0E759FF4F0C94EF2DA1
:1045A0000E948C0F55C080918F02817F8E7F8093F7
:1045B0008F0281E08093B40208950E94DB0348C01B
:1045C00080918F02982F9095917090FB80F9809345
:1045D0008F0291113DC0897F877F10C080918F022B
:1045E00081FB222720F991E0922790FB81F98093AB
:1045F0008F02992369F180918F02816080938F02ED
:1046000027C080918F0282FB222720F991E0922718
:1046100090FB82F9ECCF80918F0283FB222720F957
:1046200091E0922790FB83F9E2CF0E94A808809145
:10463000E60287FB222720F991E0922790FB87F979
:104640008093E60205C0895301C08D510E94AD22BE
:1046500081E0089580E0FACF80E0089580E0089539
:104660000C942E23CF93C82F8091B402813069F02F
:1046700038F08230C1F58C2F0E942B2281E039C0A6
:104680000E94FB0D823289F504C00E94FB0D82322C
:1046900061F48C2F0E943023811104C08C2F0E9462
:1046A000C4221FC081E090E01CC08C2F0E942E23EA
:1046B000811116C0C43189F058F4CB3089F0C03173
:1046C000B1F482E08093B40288E30E942B2208C0F8
:1046D000C93219F0C83321F00AC01092B40207C0E1
:1046E00081E0817006C01092B40280E002C080E0D8
:1046F000F8CFCF910895CF93DF9386319C4541F554
:10470000EB010E94FB0D982F8A81209102013091CC
:104710000301882379F09A7A81E009F480E080939C
:10472000B502911102C069E201C065E3C9010E94AE
:1047300071250AC08091B502811102C069E201C0F1
:1047400065E3C9010E947C250E943D0E80E001C006
:1047500081E0DF91CF9108950F931F93CF93DF9363
:10476000C42FD22FFC0182818823C9F04093B80264
:104770000E9435269093B7028093B60280E28C0F98
:10478000883008F057C0C77081E001C0880FCA9513
:10479000EAF7DF91CF911F910F910C94050680915C
:1047A000B802481330C08091B6029091B7020E94BF
:1047B0004D26883C910538F510E21D0FCD17B9F054
:1047C00080E28C0F883040F4C77081E001C0880F10
:1047D000CA95EAF70E940C06183028F581E09D2F53
:1047E000977001C0880F9A95EAF70E940506802FFE
:1047F0000E94FC051830F0F4D77081E001C0880FEA
:10480000DA95EAF70AC080E28C0F883098F4C77016
:1048100081E001C0880FCA95EAF7DF91CF911F911F
:104820000F910C940C06802FDF91CF911F910F9167
:104830000C94FC05DF91CF911F910F9108950F9378
:104840009C01CB01243F4CE5340731F188F4293D2C
:10485000FCE53F07D9F02A3D4CE5340779F1283DC6
:104860003C45A9F506E221EE41EE68ED7CE52BC062
:10487000263FFCE53F07E1F0A8F0273F3C4539F52E
:1048800007E225EE46EE67EF7CE51DC007E225EE68
:1048900045EE69ED7CE517C006E221EE40EE64EFDF
:1048A0007CE511C007E225EE44EE65EF7CE50BC028
:1048B00006E221EE42EE66EF7CE505C008E221E06B
:1048C00045EE6AED7CE50E94AC2380E008C0FC0167
:1048D0008281882319F01092B80201C081E00F9103
:1048E00008959093C9018093C80108959093BE02E2
:1048F0008093BD020895E091BD02F091BE02309711
:1049000021F00190F081E02D099480E00895E0917C
:10491000BD02F091BE02309799F020912D01222323
:1049200059F02091E60227FF07C0DC012C91119677
:104930002C93119726E02C930280F381E02D0994AB
:104940000895E091BD02F091BE02309739F022E067
:10495000DC012C930480F581E02D099408952091C9
:10496000BB023091BC022817390771F09093BC024A
:104970008093BB02E091BD02F091BE02309721F01E
:104980000680F781E02D099408952091B9023091B5
:10499000BA022817390771F09093BA028093B902CE
:1049A000E091BD02F091BE02309721F00084F185C4
:1049B000E02D09940895FC01329680912D01882301
:1049C00031F08091E60287FF02C09EE101C096E0CF
:1049D00080E0915028F021912223D9F38F5FF9CF05
:1049E0000895662351F120912D012223E9F02091B1
:1049F000E60227FF19C0462F4695469546954E314B
:104A0000E0F4677021E030E002C0220F331F6A95A6
:104A1000E2F7FC01E40FF11D828190E028233923A5
:104A200081E0232B69F409C0FC013296089621919C
:104A3000621729F0E817F907D1F780E0089581E0BF
:104A400008959C01FC0132969FEF80E0419146174A
:104A500089F09F3F19F4411101C0982F8F5F863074
:104A6000A9F79F3F39F0F901E90FF11D97FDFA957C
:104A70006283089508959C012A5F3F4FFC014281A3
:104A8000461301C01282019682179307B9F7089561
:104A9000262F2695269526952E3168F4FC01E20FE7
:104AA000F11D677021E030E001C0220F6A95EAF73E
:104AB0008281282B22830895262F269526952695D8
:104AC0002E3170F4FC01E20FF11D677021E030E03F
:104AD00001C0220F6A95EAF720958281282322835C
:104AE000089520912D01222329F02091E60227FD2F
:104AF0000C9448250C94212520912D01222329F086
:104B00002091E60227FD0C945C250C943B25209116
:104B10002D01FC013296222331F08091E60287FFBD
:104B200002C08EE101C086E0DF011D928A95E9F79F
:104B3000089508950C94992583E08093BF020C9406
:104B40009A25811102C081E001C082E08093BF02FA
:104B50000C949A250C94A12581E08093BF020C94BB
:104B60009A250C94AC2508950C94B3250C94B42587
:104B70000C94B3250C94B3250C94B325CF930E94C9
:104B8000BA250E9498130E94B825C0E08C2F0E947D
:104B9000C212892B29F4CF5FC530C1F780E001C074
:104BA00081E0CF91089508951F920F920FB60F9252
:104BB00011248F939F93AF93BF938091C002811173
:104BC00013C080912C0390912D03A0912E03B091DE
:104BD0002F034196A11DB11D80932C0390932D03AB
:104BE000A0932E03B0932F03BF91AF919F918F910C
:104BF0000F900FBE0F901F90189580913403843052
:104C000031F10E944A041092C00220E488E190E051
:104C10000FB6F894A895809360000FBE20936000B3
:104C200083B7817F846083BF83B7816083BF7894BB
:104C3000889583B78E7F83BF0FB6F894A89580912F
:104C40006000886180936000109260000FBE08953C
:104C50000E94A8080C94530482E084BD93E095BDA3
:104C60009AEF97BD80936E0008952FB7F8948091C6
:104C70002C0390912D03A0912E03B0912F032FBFF1
:104C800008952FB7F89460912C0370912D038091B3
:104C90002E0390912F032FBF08959C014FB7F894D6
:104CA00080912C0390912D03A0912E03B0912F039E
:104CB0004FBF821B930B089578941F920F920FB6EB
:104CC0000F9211248F939F93AF93BF9380912C03E6
:104CD00090912D03A0912E03B0912F030196A11D59
:104CE000B11D80932C0390932D03A0932E03B093BA
:104CF0002F03BF91AF919F918F910F900FBE0F9097
:104D00001F90189581E08093E00080E28093D800A6
:104D10001092C9008FE19EE40197F1F700C00000F6
:104D200087E090EBDC0180933D0390933E03A093DA
:104D30003F03B09340039CE088E10FB6F894A89538
:104D4000809360000FBE90936000FFCF8091E402DB
:104D50000895089522E02093E9002FEF3091E800B4
:104D6000215035FD06C035ED3A95F1F700002111CF
:104D7000F5CF2091E80025FF0BC040E050E066E051
:104D800070E00E94E9288091E8008E778093E80027
:104D90000895CF93DF9320912D01222339F02091A4
:104DA000E60227FF03C060E222E002C068E021E0E3
:104DB0002093E9002FEF3091E800215035FD06C027
:104DC00035ED3A95F1F700002111F5CF2091E8007B
:104DD00025FF1DC0EC0180912D01811105C040E02F
:104DE00050E068E070E003C070E040E050E0CE01C9
:104DF0000E94E9288091E8008E778093E80080E2A5
:104E0000FE01A4ECB2E001900D928A95E1F7DF91EA
:104E1000CF9108958093C1027093C3026093C20240
:104E200080913403843001F582E08093E9008FEFB4
:104E30009091E800815095FD06C095ED9A95F1F7A7
:104E400000008111F5CF8091E80085FF0DC040E0A2
:104E500050E063E070E081EC92E00E94E9288091EC
:104E6000E8008E778093E8000895BC0184E00C94FC
:104E70000A27BC0183E00C940A2780913303811137
:104E800009C00E947A2A0E94D72A8091E200846099
:104E90008093E20008951092330308950C94B12595
:104EA0006091300381E0611101C080E00C949C2589
:104EB0009091340381E0943009F080E060913003F8
:104EC0000C94A12542E061EC81E00E94F32942E2CA
:104ED00061EC82E00E94F3299091340381E09430E8
:104EE00009F080E0609130030C94AA25809136038C
:104EF000833009F461C030F4813071F0823009F4FC
:104F00009AC008958A3009F486C08B3009F46CC0C9
:104F1000893009F0A8C020C080913503813A09F09A
:104F2000A2C08091E800877F8093E80080913903D8
:104F300090913A03892B21F460E284EC92E003C063
:104F400060E080E090E070E00E9434298091E80009
:104F50008B778093E800089580913503813209F0C2
:104F600082C08091390390913A03029708F07BC088
:104F70008091E800877F8093E8008091E80082FDBF
:104F800005C0809134038111F8CF6DC02091F300EA
:104F90008091F20090E0922B029731F48091F10021
:104FA000813011F0863021F48091F1008093E40289
:104FB0008091E8008B7753C080913503813A09F0E6
:104FC00052C08091390390913A03892B09F04BC06C
:104FD0008091E800877F8093E8008091E80080FF5F
:104FE000FCCF80912D0136C0809135038132D9F5F7
:104FF0008091390390913A03892BA9F58091E800BB
:10500000877F8093E8000E94282A8091370380934D
:105010002D010C94A80880913503813221F58091EF
:10502000E800877F8093E8000E94282A8091380357
:105030008093E502089580913503813AA1F480912F
:10504000E800877F8093E8008091E80080FFFCCF34
:105050008091E5028093F1008091E8008E77809343
:10506000E8000C94282A089584B7877F84BF0FB680
:10507000F894A895809160008861809360001092F8
:1050800060000FBE90E080E80FB6F8948093610056
:10509000909361000FBE0C94AC250E947A2A0E9466
:1050A000D72AE2EEF0E080818460808378940C94CB
:1050B0006C2D81E291E00C9476248091340385304C
:1050C000A9F480913403853079F40E94FD25809104
:1050D00032038823B1F30E94BE25882391F30E94F6
:1050E000D3280E94A808EDCF0C942826089508958F
:1050F0000C947A28292F332723303105C9F060F426
:105100002130310581F02230310509F044C08BE3B4
:1051100090E021E535E043C021323105E1F0223253
:10512000310549F138C082E190E02CE835E037C024
:1051300099278130910549F028F0029761F5E3E164
:10514000F5E005C0EDE4F5E002C0E5E2F5E08491AC
:1051500090E09F0124C06115710541F06130710537
:10516000D1F489E090E02CE735E019C089E090E0C7
:1051700023E635E014C06115710541F06130710519
:1051800051F486EB90E02EE935E009C080E490E030
:1051900024E536E004C080E090E020E030E0FA0151
:1051A00031832083089580E189BD82E189BD09B4FE
:1051B00000FEFDCF8091D8008F7D8093D800809134
:1051C000E00082608093E0008091E00081FDFCCFF0
:1051D0000895CF92DF92EF92FF920F931F93CF9398
:1051E000DF93EC018B017A010E94472A811133C0C1
:1051F000E114F10439F0F70180819181081B190B4A
:10520000C80FD91FC12CD12C0115110519F180919E
:10521000E80085FD16C08091E8008E778093E80055
:10522000E114F10449F0F70180819181C80ED91E83
:10523000D182C08285E00FC00E94472A882321F3D3
:105240000AC089918093F10001501109FFEFCF1A34
:10525000DF0ADACF80E0DF91CF911F910F91FF90AD
:10526000EF90DF90CF90089520913B0330913C0365
:105270002617370748F06115710539F42091E800C9
:105280002E772093E80001C0B901FC0120E06115F0
:10529000710579F1809134038823F1F18530F1F1C2
:1052A0008091E80083FD3CC08091E80082FD2EC023
:1052B0008091E80080FFEBCF2091F3008091F20015
:1052C00090E0922B6115710551F08830910538F40A
:1052D00021912093F100615071090196F3CF21E0F3
:1052E000089709F020E08091E8008E778093E8002D
:1052F000CECF2111CFCF0AC080913403882361F033
:10530000853061F08091E80083FD0AC08091E8005B
:1053100082FFF2CF80E0089582E0089583E008954F
:1053200081E0089520913B0330913C032617370715
:1053300048F06115710539F42091E8002E7720932B
:10534000E80001C0B901FC0120E06115710591F18F
:1053500080913403882309F440C0853009F43FC0AC
:105360008091E80083FD3DC08091E80082FD2FC060
:105370008091E80080FFE9CF2091F3008091F20056
:1053800090E0922B6115710559F08830910540F439
:1053900024912093F1003196615071090196F2CF6A
:1053A00021E0089709F020E08091E8008E77809353
:1053B000E800CBCF2111CCCF0AC0809134038823E1
:1053C00061F0853061F08091E80083FD0AC0809132
:1053D000E80082FFF2CF80E0089582E0089583E044
:1053E000089581E00895982F973068F59093E9002B
:1053F000981739F07091EC002091ED005091F00079
:1054000003C0242F762F50E021FD02C09F5FECCF18
:105410003091EB003E7F3093EB003091ED003D7F0B
:105420003093ED003091EB0031603093EB007093DE
:10543000EC002093ED005093F0002091EE0027FD4A
:10544000E5CF80E008958F708093E90081E00895B2
:105450008091350387FF11C08091E80082FD05C06F
:10546000809134038111F8CF11C08091E8008B77CF
:105470000BC080913403882349F08091E80080FFBD
:10548000F8CF8091E8008E778093E800089520910E
:10549000E4003091E50095E64091EC00842F8170A6
:1054A00040FF23C08091E80080FD1DC0809134033F
:1054B000882399F0853099F08091EB0085FD11C02B
:1054C0004091E4005091E5002417350729F39150ED
:1054D00011F09A01E1CF84E0089582E0089583E01D
:1054E000089581E0089580E008954091E80042FF2A
:1054F000DDCF08950E94E82A0E94F02AE0EEF0E055
:10550000808181608083E8EDF0E080818F77808307
:1055100019BCA7EDB0E08C918E7F8C9380818F7E3B
:1055200080831092330308950F931F93CF93DF93DB
:105530000E94E82A0E94F02AC8EDD0E088818F7787
:10554000888388818068888388818F7D888319BC5F
:1055500010923403109230031092320310923103F0
:1055600000EE10E0F80180818B7F8083888181606C
:10557000888342E060E080E00E94F329E1EEF0E001
:1055800080818E7F8083E2EEF0E080818160808385
:10559000808188608083F80180818E7F808388810C
:1055A00080618883DF91CF911F910F910895E8ED7D
:1055B000F0E080818F7E8083E7EDF0E08081816084
:1055C000808384E082BF81E0809333030C94942A2B
:1055D000E8EDF0E080818E7F80831092E2000895F4
:1055E0001092DA001092E10008951F920F920FB608
:1055F0000F9211242F933F934F935F936F937F9359
:105600008F939F93AF93BF93EF93FF938091E100AC
:1056100082FF0BC08091E20082FF07C08091E10011
:105620008B7F8093E1000E946B2D8091DA0080FFD8
:105630001FC08091D80080FF1BC08091DA008E7F50
:105640008093DA008091D90080FF0DC080E189BD90
:1056500082E189BD09B400FEFDCF81E0809334036F
:105660000E943D2705C019BC109234030E944B27AD
:105670008091E10080FF19C08091E20080FF15C099
:105680008091E2008E7F8093E2008091E200806151
:105690008093E2008091D80080628093D80019BC8A
:1056A00085E0809334030E9450278091E10084FFBD
:1056B00030C08091E20084FF2CC080E189BD82E18E
:1056C00089BD09B400FEFDCF8091D8008F7D809305
:1056D000D8008091E1008F7E8093E1008091E2000C
:1056E0008F7E8093E2008091E20081608093E200EF
:1056F00080913003882311F084E007C08091E3009B
:1057000087FD02C081E001C083E0809334030E94E2
:1057100058278091E10083FF29C08091E20083FF38
:1057200025C08091E100877F8093E10082E0809333
:105730003403109230038091E1008E7F8093E1006A
:105740008091E2008E7F8093E2008091E200806190
:105750008093E20042E060E080E00E94F3298091C3
:10576000F00088608093F0000E944E27FF91EF9137
:10577000BF91AF919F918F917F916F915F914F9169
:105780003F912F910F900FBE0F901F9018951F9271
:105790000F920FB60F9211242F933F934F935F9365
:1057A0006F937F938F939F93AF93BF93CF93DF9329
:1057B000EF93FF93C091E900CF708091EC00D82F58
:1057C000D17080FDD0E81092E9008091F000877FD1
:1057D0008093F00078940E940B2C1092E900809145
:1057E000F00088608093F000CD2BCF70C093E9006B
:1057F000FF91EF91DF91CF91BF91AF919F918F91E9
:105800007F916F915F914F913F912F910F900FBEBC
:105810000F901F9018951F93CF93DF93CDB7DEB7EE
:10582000AA970FB6F894DEBF0FBECDBFE5E3F3E055
:105830008091F100819323E0ED33F207C9F70E94D4
:1058400076278091E80083FF2EC1809135039091E7
:105850003603492F50E04A30510508F024C1FA01BF
:10586000E855FF4F0C94EF2D803821F0823809F075
:105870001AC108C08091310390913203992389F0B5
:1058800082600FC0809139038F70873008F00BC1A0
:105890008093E9008091EB0085FB882780F91092C6
:1058A000E9009091E800977F9093E8008093F100E1
:1058B0001092F100D1C0282F2D7F09F0F4C0882369
:1058C00019F0823061F0EFC080913703813009F028
:1058D000EAC0933009F080E0809332032EC08091BB
:1058E000370381112AC0809139038F702FEF280F61
:1058F000263008F0D8C08093E9002091EB0020FF0B
:105900001CC0933021F48091EB00806214C0909110
:10591000EB0090619093EB0021E030E0A90102C020
:10592000440F551F8A95E2F74093EA001092EA006F
:105930008091EB0088608093EB001092E9008091E9
:10594000E800877F8093E8000E94282AACC081117C
:10595000AAC0109137031F778091E3008078812BD4
:105960008093E3008091E800877F8093E8000E94A5
:10597000282A8091E80080FFFCCF8091E3008068B6
:105980008093E300111102C082E001C083E08093A4
:10599000340389C08058823008F085C08091370375
:1059A000909138038C3D53E0950779F583E08A8325
:1059B0008AE289834FB7F894DE01139620E03EE037
:1059C00051E2E32FF0E050935700E49120FF03C031
:1059D000E295EF703F5FEF708E2F90E0EA3010F0AD
:1059E000C79601C0C0968D939D932F5F243149F7D0
:1059F0004FBF8091E800877F8093E8006AE270E003
:105A0000CE0101960E94342916C06091390370912D
:105A10003A03AE014F5F5F4F0E947828BC01892B8B
:105A200009F441C09091E800977F9093E800898144
:105A30009A810E9492298091E8008B778093E800F8
:105A400032C0803881F58091E800877F8093E8003C
:105A5000809130038093F1008091E8008E7772CFBF
:105A6000811121C0809137039091380399270297C3
:105A7000D4F48091E800877F8093E8008091370319
:105A8000809330030E94282A80913003811106C040
:105A90008091E30087FD02C081E001C084E0809333
:105AA00034030E9462278091E80083FF0AC080913E
:105AB000E800877F8093E8008091EB00806280930C
:105AC000EB00AA960FB6F894DEBF0FBECDBFDF91F4
:105AD000CF911F9108950895CF9380913403882327
:105AE000A1F0C091E900CF709091EC00892F8170F6
:105AF00090FD80E8C82B1092E9008091E80083FDBA
:105B00000E940B2CCF70C093E900CF910895DB0168
:105B10008F939F930E94132EBF91AF91A29F800DF0
:105B2000911DA39F900DB29F900D1124089587FBA6
:105B3000082E062687FD819567FD61950E94262E19
:105B40000EF4919507FC81950895AA1BBB1B51E1AA
:105B500007C0AA1FBB1FA617B70710F0A61BB70BDD
:105B6000881F991F5A95A9F780959095BC01CD0182
:105B7000089597FB072E16F4009407D077FD09D0FF
:105B80000E94A52D07FC05D03EF4909581959F4F6E
:105B90000895709561957F4F0895A1E21A2EAA1B72
:105BA000BB1BFD010DC0AA1FBB1FEE1FFF1FA217CD
:105BB000B307E407F50720F0A21BB30BE40BF50BCA
:105BC000661F771F881F991F1A9469F76095709553
:105BD000809590959B01AC01BD01CF010895EE0F1A
:105BE000FF1F0590F491E02D09940E94FD2D3323B1
:105BF00012F48A1B9B0B0C940E2EA29FB001B39F34
:105C0000C001A39F700D811D1124911DB29F700DC5
:105C1000811D1124911D08950E94FD2DB7FF089547
:105C2000821B930B08950E94FD2DA59F900DB49F9C
:105C3000900DA49F800D911D11240895B7FF0C9421
:105C4000132E0E94132E821B930B0895991B79E04B
:105C500004C0991F961708F0961B881F7A95C9F7FC
:105C600080950895FC014150504030F00190061697
:105C7000D1F73197CF010895882799270895FB011F
:105C8000DC0104C08D910190801921F441505040F5
:105C9000C8F7881B990B0895F999FECF92BD81BD75
:105CA000F89A992780B50895A6E1B0E044E050E065
:105CB0000C94862EA8E1B0E042E050E00C94862ED1
:105CC000262FF999FECF92BD81BDF89A019700B4B5
:105CD000021639F01FBA20BD0FB6F894FA9AF99A55
:105CE0000FBE08950396272F0E94612E0E94602EFA
:105CF000252F0E94612E242F0C94612E0196272FB0
:105D00000E94612E0C94602EDC01CB01FC01F999FC
:105D1000FECF06C0F2BDE1BDF89A319600B40D92F7
:0C5D200041505040B8F70895F894FFCFB0
:105D2C00C8005B02280850011E0A14010101020080
:105D3C000E000E0E01191A1B1C1D1E1F20212206FF
:105D4C0001A626C926AA2639273527A92601E2004D
:105D5C00E900EA00B500B600B700CD008301CC0025
:105D6C008A019201940121022302240225022602B7
:105D7C0027022A02B300B4006F007000818283E214
:105D8C0000E900EA00B500B600B700CD008301CCF5
:105D9C00008A019201940121022302240225022689
:105DAC000227022A02B300B4006F007000818283C4
:105DBC00F4F7F5F667663635349796949593313249
:105DCC0033F0F10001020202020606060909090974
:105DDC0009090F0F0F0F0F0F151515181919191990
:085DEC001919191919192324D2
:00000001FF
